:100000000C942A001895000018950000189500001F
:10001000189500001895000018950000189500002C
:100020001895000018950000189500000C947000B9
:10003000189500001895000018950000189500000C
:1000400018950000189500001895000018950000FC
:10005000189500008FE58DBFC0E4E8E34E2E84E0E4
:100060008EBFD4E0F4E05F2EEEEFF3E0A0E6B0E068
:1000700088278D933197E9F780EA89B981E080BDBF
:1000800088E18AB984B7082E877F84BF8FE181BD5C
:1000900087E081BD0E94160166248CE00E94640105
:1000A0000E940B017894579AB89AC0980E94070151
:1000B000EAE7F3E00E940001E6E8F3E00E94F200C4
:1000C0000E94F900A3E6B0E088278C93A3E6B0E095
:1000D0000E94EC000E94F9000C946600F894FFCF97
:1000E0000F921F922F923F924F925F927F92AF9208
:1000F000BF920F931F932F933F934F935F936F93F1
:100100007F938F939F93AF93BF93CF93DF93EF939F
:10011000FF938FB78F93A0E6B0E08CB18C93A0E6ED
:10012000B0E08C91A1E6B0E08D9388278C93A1E696
:10013000B0E0EEE8F3E00E94A90111F00C94A800F1
:10014000E1E6F0E0A3E6B0E00E94A4010C94B00068
:10015000E1E6F0E0A3E6B0E00E94E3000E94A40123
:10016000A3E6B0E0E0E9F3E00E94A90111F00C94ED
:10017000C70088B391E0892788BB0E940B01E6E99C
:10018000F3E00E940001A3E6B0E088278C938F91F2
:100190008FBFFF91EF91DF91CF91BF91AF919F9171
:1001A0008F917F916F915F914F913F912F911F910F
:1001B0000F91BF90AF907F905F904F903F902F90A6
:1001C0001F900F9018958F938D918823E9F71197C1
:1001D0008F910895A0E2B4E08D91882311F00CD0A6
:1001E000FBCF08950E94A001802D11F005D0FACF19
:1001F00008958DE001D08AE05D9BFECF8CB9089513
:100200000E94A001802D11F059D0FACF089582E00C
:100210005BD009D005C081E057D005D080E854C03C
:1002200080E852D0089583E099277BC08AEF90E060
:100230000E9491018F9A8E9A8D9A8C9A8B9A8A9AA3
:10024000929885E090E00E949101939897989698F3
:10025000959A949A939AEF93FF93E4ECF0E00E94BE
:100260008501FF91EF91939859D0939AEF93FF9363
:10027000E4ECF0E00E948501FF91EF9193984ED05D
:10028000939AEF93FF93E4ECF0E00E948501FF91D5
:10029000EF91939843D09498939AEF93FF93E4EC63
:1002A000F0E00E948501FF91EF91939837D088E2AA
:1002B0000BD08EE009D086E007D00895929A8295FF
:1002C00005D004D02BD008959298F9CF859510F4DD
:1002D000949A01C09498859510F4959A01C09598C8
:1002E000859510F4969A01C09698859510F4979A82
:1002F00001C09798939AEF93FF93E4ECF0E00E948B
:100300008501FF91EF91939808953197F1F7089542
:10031000689462F80895E89462F8089581E090E0A6
:1003200000C0EF93FF93EE27E82BE92B31F0E0EDCF
:10033000F7E03197F1F70197D1F7FF91EF91089529
:10034000C89531960020089581918D938823E1F717
:100350000895689401C0E894AF93BF938D9116F00F
:10036000919103C00E94A001902D891718F011F4FB
:100370008823A1F7BF91AF9108955072696D696F9D
:100380002073616D3A00697266616761000049001F
:10039000497266616E005072696D6C6A656E6F00BD
:00000001FF
